:10000000C128B000F839A400A40CA40C240C840767
:100010006C20B0000005BC283008031C030100065A
:1000200030058006BC28A01123080319A01505304F
:10003000A2002730A900103029200330A900E830A1
:100040002920A90164302920A9010A3029202A0881
:100050003028A8002B08A5002A08A400792024082D
:10006000A400A2030319A011230803193A282202AD
:10007000031841282408031DA011A0194128303E6F
:10008000472808000C1E422899000314BC28211997
:1000900042280800A901A800FF30A807031CA907EF
:1000A000031CBC280330A500E53058204C28A501CE
:1000B000F63EA400A509031C6328FE300000A40737
:1000C00003185E28A4070000A50F5D28000024186F
:1000D000692824186B28080000308A003008073986
:1000E000820701340234043408341034203440349C
:1000F0008034AB01AA011030AE00250DAA0DAB0D66
:100100002808AA022908031C290FAB0203188F280C
:100110002808AA0729080318290FAB070310A40D04
:10012000A50DAE0B7D282408BC281030B100A50118
:10013000A401AF0CAE0C031CA3282808A4072908AF
:100140000318290FA507A50CA40CAB0CAA0CB10B26
:1001500099282A08BC28A400A71BB0202408BC2882
:10016000A409A509A609A709A40A0319A50A031940
:10017000A60A0319A70A08008313831203130000B9
:10018000080083160F3099002030980083128030C9
:100190009800A001C23083168600FD30850007302C
:1001A00083129F00BC2986156430572006146430E2
:1001B00057208611643057200610643057200800FD
:1001C0008615851464305720861126213821061B98
:1001D0001D2985190B294D304220413042204730DE
:1001E00042204E30422045304220543042203D30A3
:1001F0004220203042200430A100A3013508AB008A
:100200003408AA00132020304220422042204220FD
:100210000D3042201C294D303407BC00350803182E
:10022000013EBD004D3042203408422035084220B6
:100230003C0842203D084220E728E02885100A308B
:100240005720080085140A30572008000930BB00E9
:100250001E212221343084003B08003E012003107F
:10026000051803140C200130BB02031828290800CC
:100270001E21222183100518831483183A14831C2D
:100280003A101E2122218310051883148318BA14F2
:10029000831CBA101E212221831005188314831891
:1002A0003A15831C3A111E2122218310051883144C
:1002B0008318BA15831CBA111E2122218310051838
:1002C000831483183A16831C3A121E2122218310AC
:1002D000051883148318BA16831CBA1286151430B5
:1002E000572008003508AF003408AE00A9012D30B2
:1002F000A8009520C0002B08C1004008BE0041089E
:10030000BF000730A4000310BF0CBE0CA40B832950
:100310007F304005C200C3014308AF004208AE0071
:10032000A9010A30A8009520C2002B08C30042088A
:10033000C4004308C5000730A4000310C50CC40C5A
:10034000A40B9D297F304205C000C101C108031DD7
:10035000AD2940304002031CBB294408093A45043A
:10036000031DB829BE0A0319BF0AC501C401BB2970
:10037000C40A0319C50A080006100330A900E830B2
:100380004B20C801C701C60186158514B501B4010B
:10039000143057200519CE29D320E02886111430B7
:1003A000572026218618F9293508AB003408AA0001
:1003B000AC01AD01013EB600FC30B7002B080318BC
:1003C0002B0FB707FF30B8002C0803182C0FB80705
:1003D000FF30B9002D0803182D0FB9073908A70001
:1003E0003808A6003708A5003608AB20B400250859
:1003F000B50002304802031C092A4708A500460838
:10040000A400A9014808A8007920CA002508CB004B
:100410000D2A4708CB004608CA0035084B02031CCA
:10042000202A031D172A34084A02031C202A3408F4
:100430004A02CC003508031C013E4B02CD00282A9D
:100440004A083402CC004B08031C013E3502CD00A3
:10045000CD08031D2F2A04304C02031C362A350810
:10046000C7003408C6000130C800412A0F304802D6
:100470000318412A3408C60735080318013EC70788
:10048000C80A382101304A20BA1D482A06124A2AD1
:10049000061606163A1E4E2A8612502A861686160A
:1004A000061B9E2A85197E2A7221413042205A302D
:1004B0004220493042204D304220553042205430B5
:1004C000422048304220203042203D30422020301F
:1004D00042200430A100A3013F08AB003E08AA005F
:1004E00013202E304220A3014508AB004408AA0087
:1004F0001320203042200D3042209B2A41304607F5
:10050000B20047080318013EB30048083207BC0098
:1005100033080318013EBD00413042204608422006
:1005200047084220480842203C0842203D0842201B
:10053000C801C701C601061B9E2A9B2AC429630065
:020540009F2AF0
:02400E00223F4F
:00000001FF
